S01100004D49432D5765656B322E737265634F
S113000045C0000061C0000090C00000C1C00000F5
S11300105AC0000064C0000056C0000054C0000074
S113002052C0000050C000004EC000004CC0000090
S11300304AC0000048C0000046C0000044C00000A0
S113004042C0000040C000003EC000003CC00000B0
S11300503AC0000038C0000036C0000034C00000C0
S113006032C0000030C000002EC000002CC00000D0
S11300702AC0000028C0000026C0000024C00000E0
S113008022C0000020C000001EC0000011241FBEBA
S1130090CFEFD0E1DEBFCDBF11E0A0E0B1E0ECE2F4
S11300A0F2E000E00BBF02C007900D92A031B1074F
S11300B0D9F721E0A0E1B1E001C01D92A231B2075D
S11300C0E1F7B1D0B1C09CCF1F920F920FB60F923F
S11300D01124959A0F900FBE0F901F9018951F92A0
S11300E00F920FB60F9211248F939F9393B181E0D7
S11300F0892783B99F918F910F900FBE0F901F9006
S11301001895892B21F085B3869585BB03C085B3EB
S1130110880F85BBAF9B03C081E085BB089585B381
S1130120811102C080E885BB08951F920F920FB61B
S11301300F9211240BB60F922F933F934F935F931B
S11301406F937F938F939F93AF93BF93EF93FF939B
S11301508091100190911101009711F4959805C0B8
S1130160019719F481E090E0CCDFFF91EF91BF910A
S1130170AF919F918F917F916F915F914F913F913B
S11301802F910F900BBE0F900FBE0F901F901895DC
S11301901F920F920FB60F9211240BB60F922F934A
S11301A03F934F935F936F937F938F939F93AF93FB
S11301B0BF93EF93FF9380E090E0A3DFFF91EF9173
S11301C0BF91AF919F918F917F916F915F914F916B
S11301D03F912F910F900BBE0F900FBE0F901F9069
S11301E0189514BA8FEF81BB80E090E0A0E0B1E0F5
S11301F023B3213011F4019601C023B3803191055A
S11302002CF01E962C911E9722BBF2CF99232CF42E
S11302101E962C911E9722BBEBCFFC01E050FF4FA2
S10F0220208122BBE5CFDDDFF894FFCF86
S113022C3F065B4F666D7D077F6F777C395E797116
S9030000FC
